:100000000C946600189518951895189518951895DC
:100010001895189518951895189518951895189578
:100020001895189518951895189518951895189568
:100030001895189518951895189518951895189558
:100040001895189518951895189518951895189548
:100050001895189518951895189518951895189538
:100060001895189518951895189518951895189528
:100070001895189518951895189518951895189518
:10008000189518951895189518951895809BFECF7A
:100090008099FECF08950C9BFECF0C99FECF08955A
:1000A0008A938EEF0FEF07BB08BB889800E002BB76
:1000B000149803B9EBDFEFDF88BB880F81608F3FB7
:1000C000D1F78EEFF8CF00008895FECF0FE30DBF7C
:1000D00001E00EBFC0E2D1E00E9474000E94500017
:0C00E0000E9463000C94630001E008958E
:00000001FF
